:2000000000080020451000007100000073000000000000000000000000000000000000007F
:200020000000000000000000000000007500000000000000000000007700000000000000D4
:20004000074500000D45000013450000194500001F450000254500002B4500003145000098
:20006000374500003D4500004345000049450000FEE7FEE7FEE7FEE7FEE70020006880F3F8
:2000800008887047000044014F637420323720323032300032323A34323A3533FE49C97A11
:2000A0004B09FD492039CA8B0243FC48002B02D0037EDB070CD08B8C1A404B8C1A434A84C0
:2000C00003D0027FFB231A4002770020C8837047CA837047F24881210180002101807047FF
:2000E00070B5F0498A88D243920706D0EA4A927F322A02D34009002303E0C200101AC00992
:2001000001233C2801D23C2002E0FF2800D9FF200A8AE54C120AC01E824215D0002B02D1C1
:20012000257B012D03D0551DA84200D928460A8A40252A430A820A8A4F26324000020243C7
:200140000A82088AA8430882237370BDD6480021803801734173D248012101800115818056
:200160000F210180022202810183042181827047F8B5CE48008B4726C004C40E3602B08A01
:200180000090318B641C411AC9480D46604304F011FAC54FC822403F78870098294650431C
:2001A00004F01EFAFF219131081AB887F58BF08A291AC048604304F0FDF980B2F887152137
:2001C0006843614304F0F6F9192180094901081A00B28D225043C217120EB349101800129B
:2001E0000880F8BD70B50546B048008BAE4CC004403C617CC00E814202D06074FFF7B8FFD4
:20020000AD48854203D83C21608F615E1FE0AA48A54A4030854203D30021E08F515E16E01A
:20022000A548618F40422B18E08F401A5843C617B60E3018801140180021515E3C22A25EB8
:20024000891A5943CB179B0E5918891189184543280C401800D5002070BD944A108BC004B5
:20026000C10E8D482030007B4000401C1F2800DD1F20814200D2481C118B1F231B02994340
:2002800000020143118387490888072212029043814A4032927A5207520D10430880704781
:2002A00082494A140B8B002805D093430B83032803D9002207E013430B830321484001215C
:2002C0004003090342187D48018807231B039943114301807047F8B54109794A00290AD0BA
:2002E000202901DB1F2106E0937C8B4201DA491E01E08B4200DD9174674F4722BE7F120295
:200300000E23B100D3561C31684AC918118223367D217043C90004F04DF93C46A034A17C3F
:20032000081A04D4E17C40434143481100E00020E18A0D18A08AA84200D205463003D2211F
:2003400004F038F91F217956401908185D49884200D908462082F8BD10B55B4A00211170F6
:200360005149012440394B7A23434B72574903888B8043880B8183888B81C0880882B42013
:2003800010704F4820381081072090804E48022220380272037972B61343037162B64B4887
:2003A0002030027AFB231A400272088810221043088010BD00B54248FB22417C11404174FC
:2003C000392138480902018281888908890081800188F022914301800020FFF761FF3349AF
:2003E000082088832C4880222038018C914301841046FFF753FE00BD314EA03E34464034D1
:20040000217A607A814201D130BFF9E7810089198D68002D0CD0401C0007000F6072A847AF
:200420000028EDD072B6284603F040FF62B6E7E703F05CFFE4E7F8B5174C203CE08B002811
:2004400002D00020FFF72AFE1D4E3221A03E3068401C306004F0AEF88446002955D1C007F2
:2004600008D11149C039486A002803D0421C01D0401E4862084D2035A87F2F464037002887
:200480002AD0401E0006000EA87725D104207873208C012108431BE020000020206C0040AC
:2004A000004C0040003400407004002000300040001A040080920800DA020000203800408C
:2004C000D0010020FF0F0000206000400044004020840846FFF7E2FDE87F0090002814D00F
:2004E0000A21604604F066F800290ED10098401E0006000EE87708D108207873208C0121AE
:20050000084320840846FFF7C9FDF84CA07B800704D472B6706803F0C9FE62B6A07B4007F0
:2005200009D5F348817DC07D814204D072B6F14803F0BCFE62B672B6B06F03F0B7FE62B6A3
:200540000020F8BD10B5EC4C207A800702D5EB4803F0ACFE0720207210BDE948E94A01898D
:20056000511A0022825E8818704770B5DF49487A0C46403C002820D00025032805D0022873
:2005800006D0012804D04D7222E003F03AFC07E001F07FFF0420D649E072DB48603948604F
:2005A000D348202220388572D0486038018C114301841046FFF772FD0AE0D4480179C9076E
:2005C00006D00079C00603D40220E072D0488047002070BD00B5CF4800228280CD49403118
:2005E0000A74CD490180C948082140388183CB490183CB4981200880CA4909200870FFF7B1
:2006000069FDBB49C84860394860C8480178490849000170B5484038C2722038018C2522B6
:20062000520111430184A020FFF738FD002000BDBC480178422211430170BD49C0140860DE
:20064000BC49086070470188428851188288C08851184018AA4900228A5E8010801A00D5AB
:200660000020704770B5A24D0023603D0AE04400641980342488260B964207D12405240D89
:20068000E31840180828F2D3184670BDAA4870BD70B5022211460020FFF7E4FFA74C944DFB
:2006A000217B603D49000326800349193602000C89198882012204211046FFF7D3FF217BB8
:2006C000C00349004919000C89198884032208211046FFF7C7FF217B042249004919891983
:2006E000888308210720FFF7BDFF80492039C880207B401C8007800F207313D120460C3855
:20070000FFF7A1FF79491F2240318A560B468018A03B9885201DFFF796FF1886201FFFF773
:2007200092FFD88585482038417A490849004172002070BD10B57A49302008766C48002225
:200740004030837E002B0CD00446203CE48E0C82047E0C75012B02D003F075FC10BD827651
:2007600010BD01230B8002736A48018A0C229143018210BD014610B56A480089704A401C9C
:20078000504303F017FF594980B220394881BE2801D9602010BD462801D8002010BD202046
:2007A00010BD524910B52039CA8AC0075400C00F04436248CC822038817B491CC9B281730E
:2007C0000C2908D3200903F07AFE2107090F884201D1012010BD002010BDFEB5444E032056
:2007E000603E424C00023018603C00902046C03001900B204B4F800135183878400605D40E
:20080000608E002804D13068012801D90020FEBD30680F2868D2297B687B8142EDD0410026
:200820008A190521C901401C51180007098D000F6873288A8C46401C80B22882042854D9C4
:200840006046698142002981002359000919C031098A68898A18814201D2698103E0288953
:20086000814200D929815B1C062BEED30199097F491CCBB20199062B0B7702D3019B0021E6
:20088000197701996046097F49000919C03108821648052140308277D0086086C901401A4B
:2008A000A12802D300202882A7E72B896889191A0E297DD9009A00211173C0184108907C71
:2008C00061454CD900283FD0907A00283CD0D17C002901D1022835D90020D0740120FFF7DD
:2008E00060FF002854D12FE06AE072E06000002090010020F9420000005400403704000066
:20090000204700003104000055240000403000400110002000340040010A00003B3B0000EC
:2009200000380040003C00406B050000406C004080E200E000E100E0FFFF000050040020F2
:20094000701700000120D074009900208872C97A491CCAB20099CA7227E088744DE70028A0
:2009600006D0D07A002818D0D17C00290AD107E0012090740020D0749073FFF712FF0CE090
:20098000022808D90020D074FFF70BFF002804D06020FEBD0CE00120D07400990020C8726D
:2009A000897A491CCAB200998A72052AD6D9D4E700980099007B401CC0B20873282803D904
:2009C000608EFFF7D7FEE4E7002088748872C87213E702280DD0002160464A001219C03214
:2009E000491C10820629F8D3009900208874087303E708466186FFF7BDFEFE484089C0082F
:200A0000401E3881F9E6FC4801210170812101703B2101710F2101812121017070471CB53B
:200A2000F749F6480860FFF728FBF6485A2101700025057109210172F34981810A218182E9
:200A4000F249018308218183EE49022020310876EF488580EF490180392109020182EE486F
:200A600001240480EC4981200880EB48EB4920300180EB48E8498078204320310871E9487D
:200A8000047418218182E849202008760877E6492031087008730874E44881B2E44803F0C7
:200AA00007FD3022E349E44803F0C6FA4B20000103F024FDFFF7A7FF03F00DFDFFF746FB85
:200AC000DE4906200860CE4980390860DC4804800321018041210176D6480838FFF73CFC77
:200AE000D8480571D84C6572FFF777FEC14F203FF872FFF7EFFA3846B0302021019003F01F
:200B0000D7FCD048017A8907FCD5CE4A002120321170CC4802210172072201210020FFF7F7
:200B2000A1FD4003010CB348B24D4038403D818329462E46F87A40316036C03500912028AA
:200B40003BD0602848D0FFF745FDC148BF498167C048017DA74C403C2170017C6170007E67
:200B6000A0700120BC49E07001C9606020460C22B03003F061FAB84908221031284603F0D6
:200B80005BFA4220608100990D2008730220B0720F20B87720464021E0300174FF219C31A1
:200BA000603881829E49AD4B8A889A4244D0CA88C2820A890283897A43E0A548A849416066
:200BC000A849C167A848A0649B48A84981613020F0720020F8752CE09D48A5494160A548A6
:200BE000A0649548A44981610024F4721022A349019803F021FA00984089BE2802D2A87FB4
:200C0000001DA8778448203001887322C9B212028918018080499A48888003200881A87F27
:200C200006225043C01C88814D2008800F2008820C75FFF7FDFC88E7C821C18291490183FD
:200C40008521817601250577722141770C2181770E21C177FFF781FC66496031C877FFF796
:200C600087FA78488021017087480570812101700D2101708449952220310A80FF218182A9
:200C8000032109020182002101716C49612008605B4980390860208C2021084320847B490C
:200CA000A184F97A002902D178492031A1840121890208402030FFF7F1F95F48744941603F
:200CC000FFF79AFB4B4810B54038C18C714A0A4002D0038C93430384428C464B8A434284B7
:200CE000203BDB7A1B0705D5890403D55849564B096899660021C184002A05D14A482030E9
:200D0000017F04221143017710BD10B5404800228088000700D510223A48808B0821C00495
:200D2000002800DA0A435C488389DB060CD5042380891A43800607D52E4803232038C376D6
:200D40002030C3890B43C3812A4B1C24403B188C01462040504004D0A14311431984FFF7BB
:200D60009DF910BDF0B53748027A01790A400272D1071AD00179490849000171002101745A
:200D80000170334B60335D7D3F490224052D09D00E7904252E430E710E8AC127BF00BE435E
:200DA0000E825D750B7923430B71910778D526493A4C4B7A1A0774D5254A0F6D8032168827
:200DC000BC463605360DF61997884D6D3F053F0DF61917893F053F0DF6190E65B646568880
:200DE000D7883605360D3F0576193F0DF61957893F0557E040000020003C0040FF0F0000A3
:200E000080E100E000300040051D00003B23000000340040010A000000380040103000006A
:200E20006047000060400040006C00409C04002000000020981000000001002080E200E094
:200E4000004400400060004030040020B7130000300100206058004084000000FFFF000085
:200E60009F12000091060000D342000035070000B72200008D200000AD43000044240000FB
:200E8000ED0200000E0B000000640040418700004505000021830000204800402060004088
:200EA00027E02FE03F0DF7194F65D28916056B4A360DD6805A0709D5CA6D6515521CCA65BB
:200EC000AA4217D3FA2213404B720CE066467246760A921B0A656A0ABA1A4A659A0709D5AE
:200EE0005A0852004A720179FD221140017100202070F0BDB42020705948018810221143B5
:200F00000180F0BD0179FD2211400171002020705448C06F03F0CAF9F0BDF0B5524A908A0E
:200F2000118A0840FF219182C62104464D4B0C407021C95ADD6E02266033002C25D0C424C3
:200F400020400024002808D0107930431071202003F0D4FA0620587507E0587D042803D1E0
:200F6000107B69182039C8775C7501201070032000021082FC20107714713C48047004740C
:200F80000179490849000171F0BD364CC7074034648E002F03D0200A10735E75F0BDC00673
:200FA000FCD5587D022812D021201071FF20C33010822E4840220270902202740583891E78
:200FC00081820121017202790A430271F0BD147303205875F0BD00B525490F200883254823
:200FE0008069002802D003F061F900BD0020088000BD21497F2088822048C1780A060AD4FD
:201000001D4A203A127ED20605D580221143C1701B4A02211174C17809090901891DC1706D
:20102000704700B517480178490604D541210170154803F03BF915480179C90701D0102144
:20104000017100BD082003F059FA10480178490602D50179C907F9D0FFF7E1FC40000020B6
:201060000044004030010020006400400060004000500040B0020020406C00407004002075
:2010800040340040003C0040D5050000403000400707070707070707650D00005745000050
:2010A00069450000D70F0000790000001B0F00004F45000079000000F30F00007900000071
:2010C000790000002310000010B5E848007C00F0F1F9044607281AD8E449621C1031E44896
:2010E00002F08EFFE2480C21113801740069E1490840E149884207D1DD4891380068002837
:2011000000D1401EDD494864204602F0F4FF10BDF8B5D64C8034207F2646401EC1B22177BF
:20112000D648403E0090002917D02046008C08291FD38A0710D12246C03AE38B958D5B1986
:201140009BB2E383128E801880B22084082903D11909E18300092084F8BDC079C107FBD114
:201160000007F9D50320F072707A202108437072F8BD0629FCD801212177FFF733F80546DF
:20118000BF480088000BC10705D04007800F0A21401C48434519E08B152169434843070BE8
:2011A0000020E0832084072138464907084303F061F8B4488188012904D0B3498D4203D9D1
:2011C000052005E0002003E000880006800F401C6077A64C0006C00D403C00196030017C4B
:2011E0007943CA09112141560A204143881800D50020B087009A012191719C492039897F19
:20120000322904D39949A031097C4143C8099F49884200D90846C0019D4903F0CBF905468D
:2012200099489349BA30113908828D74012002F062FFA586F8BD8E4800B5964911380161C9
:2012400041214902818200218175052002F053FF00BD874800B59049113801828349403933
:2012600049890A0A12021232428201756421417582492031097B4A00014680395218032143
:2012800009025118794A0B7D6032927F9B188375097DC1750276072002F02DFF00BDF8B55E
:2012A0007E4801782022114301700178DF2211400170724E707A002802D17948FFF74CF80C
:2012C0006B4C0F34207B002863D1E07B25460027603D00281BD0401EE073A87A032858D357
:2012E00072B6704802F0E2FF62B6207CE17B401E81424ED16148403887820782607C8006D6
:2013000047D45F48018882149143018041E07771A87A0127030003F077F90906151A313C33
:20132000343C373A3C005248913800681D2830D9082020744E48322111388164AF7202F091
:20134000A6FF26E0FFF785FF0220A87221E0474840214038028C0A430284428C0A43428481
:201360004E482038017FFB22114001771E202074FFF761FF0320A872B7710AE000F077FB40
:2013800007E000F060FD04E000F098FB01E002F01CFF0020F8BD364800B50F30417C0A07AF
:2013A00003D5F7221140417400BD082211434174FFF700F800BD70B5FFF7A7FC2B4AD4890B
:2013C000002C51D00020D081104621044030002903DA417A082319434172E10603D5417AEF
:2013E000042319434172E3070121002B02D0437A0B434372A30526D52B4B10251E78282EB4
:2014000002D15B78002B0DD0037ADE0713D00222427316484038028C0A4302840120FEF7B3
:201420003DFE10E0027A0A430272417A294341720321817207E00B4303728172417A29438F
:201440004172507FD077A00601D5FFF73BFC200702D50A48806C8047600701D5FFF7DFFA0B
:20146000A00701D5FFF797FF002070BD40000020C101002000FFFFFC0028062C300400202C
:20148000203800400034004052030000E8260000881300000C510A000C710000406C004072
:2014A000AC14000031180000000800203231320332313214202801D201207047802803D24A
:2014C00020380011801C7047E02803D28038C01008307047E0388010143070474107890F79
:2014E00003290BD1010703D58009022804D005E0000903D00C2801D8012070470020704700
:20150000F0B5FB4AFC4E107F34460025F94B803425280CD0FFF7E2FF002815D0107F217A3A
:20152000C0074907C00FC90F884237D034E0F248517F8030CF08007A002F13D0012F16D0D5
:20154000022F14D0052F01D0022014E0282018705D70E580A58022202072607AEF2108402E
:20156000607219E02021E57208432072F0BD368CB60502D50120E072F0BD1970927F490720
:201580005A70490D0423091DE3805118A18002210843FB21084021E0E572F0BDD449E08895
:2015A0004031CA7B811889B2E180A788B9420DD9607ADF210840607210206073308C01215B
:2015C000084330840846FEF769FDF0BDC84918181D3102F015FD207A042148402072DBE788
:2015E00010B5C54C208C00041CD4C1484030C17B491CC9B2C173042901D90421C173CAB2D0
:20160000BB49BD481C31583002F0FAFCBA4802228030417A11434172218C90030143218443
:20162000FEF73CFD10BD30B5B34C803461882088814202D30020A07230BD451A042D00D966
:201640000425227A2801130701D5072300E00623184308235A402272A54A20321074A54813
:201660002A460918A248313002F0CAFC608840196080A1484030017F817730BDF0B5074605
:201680009B4C89B04034A079F90100908E469A49974E4A8EB18A0191317F8007A57B8C46A9
:2016A00000285CD06046400871460843C0B23077002D0CD0072D13D302210422FF2812D058
:2016C000002845D0552845D0332845D0A3E0104648214843894902F06DFF01994018F0826A
:2016E0006D1CA573A2E0009880072FD5824D8035287B002805D0012820D0022824D003281E
:2017000024D17D4800264030C6777B49FF200A8C013002430A84FEF7C1FC287B0028687A60
:2017200004D0CF21084068722E720FE0EF2108406872287A40084000287207E06A80287ACB
:20174000F72210402872A972FFF76DFF012004E0E17160E0E2715EE00820E0715BE0644881
:201760004030C17B407B002D14D0614A1C32092D23D00A2D52D3002F4DD00023A3730028C6
:2017800038D088423AD91046891C02F042FC002838D040E0002F3ED10123A373002801D078
:2017A0000B1A9B1C5820584308305043534902F001FF01994018F08238E00A21A173805C4A
:2017C00002F030FCB84226D0A07900282ED1607B00282BD0E17B884228D3FFF701FF464818
:2017E0006021408E4843454902F0E4FEB18A4018F08210E06046FFF75DFEE073607B401C37
:20180000607313E0A079410701D51020A5E7000701D5FFF775FE012009B0F0BD815C7346AC
:20182000490819438154A07B401CA0730020F3E7F8B52F4D3248298A0026324F814209D108
:20184000E88A411EE98203D3387C401EF873F6E0FE73F4E02848264CA98A40304034009055
:20186000002909D1E6716673A6730F20E88226493F200881FEF76AFCA6E022495000A039B7
:2018800040180521C9014018018D521C1007000F6873288A401C80B22882032838D801285D
:2018A00006D06A8A511889B26982032805D105E06E82E672A672A674E67485E0491C4808FB
:2018C0000D49688248866031897BC90701D1FEF707FC698A0D4A4808801802F06BFE81B20B
:2018E000009801810448C28A91426DD9C1826BE0F0030020000800200000002070170000AD
:20190000FFFF0000D0010020003C004000DC0500F848C279062093079B0F9840801E5207C7
:201920006A8A03D51018884203D320E0101A88421DD9E07A401CC0B2E0720A2853D8A07C36
:20194000002812D0A07A052801D9002005E002280BD9E07C002806D00120FFF78FFE002823
:2019600041D1E67401E00120E074A6722CE0A07A401CC0B2A072A17C00290CD0E17C0029DF
:2019800003D005280CD9012002E00A2808D90020FFF774FE27E0E07A022801D90120A0742A
:2019A000E07A052801D9002005E002280BD9E07C002806D00120FFF761FE002813D1E6747D
:2019C00001E00120E074E672287B6A7B904200D053E7387C401EF873A88A401C80B2A8828E
:2019E000E98A88422BD9FEF775FBC3482882A6716079002801D0162000E005206071E0793E
:201A0000002801D0607911E0E88A0F2804D9A98A401A6179401809E0A88A3A7C0146001D89
:201A2000904202D2C8B2101A00E00420E882A88AE98A4218397C8A4201D2081AE8820020EF
:201A4000F8BDAC4800B50C22AC49303002F0F4FAAA49A84810220C31303802F0EDFAA54845
:201A6000142180388177A6496C20088200BD00B5FFF7E7FF9F490320A039086508468030DF
:201A8000417A0122114341729E4902224A75014620226039CA729C49816241629C499B4806
:201AA000C8819848A0380168803041640164826C891AC16305214038817200BD00B53120F9
:201AC00002F0B2FB02F093FBC1B2002002F0A1FB00BDF0B587484038807BC00601D5002066
:201AE000F0BD844883492030A039008A898D421A02D50124504201E000241046C1088448FE
:201B00000023603000290BD0C3758375082202757F2900D97F21002C00D0494248B2F0BDEE
:201B2000857DAA1856B28675C27D521CD5B2C575AA07F0D1027D964202DD0121002404E09E
:201B40005742BE4207DA01210C460C2D01D3521C02758375DCE7C375457D6D1CEDB245750E
:201B6000202DF6D94375042AF3D9521EF0E7F0B5604C6849A03CE08D85B04843000CA08712
:201B8000A08D604F4843010C20464030A03F019001803D46803538685A4EE863707C41070B
:201BA0002046C0300290002954DA208EFEF71AFB019900908880204660300390807BC007B1
:201BC00045D1608EFEF78CFA0098FEF784FBB07C042805D250498A88920709D5012206E020
:201BE000042805D94C498A88920701D403228A80FEF756FBB17C0A2901D2002008E00F29DE
:201C000001D2012004E0142901D2022000E00320414A1288F0239A43800102433E480280D4
:201C2000072901D9162100E006213B488181818802888901D20818231A4000881143400926
:201C400006221040014303980173FEF706FBFFF740FF1BE0FFF73DFF717C0A0716D40298DF
:201C6000A28D008A824205D838686A6C801A2B4A904209DB0720014371743220A864386881
:201C80002838E86305B0F0BD372007E0411D0A2902D9717C090701D5962100E03221A964C3
:201CA0001B49144B40314A6C803B002A38D03E68B21A164EB24201D900224A64134AA68D49
:201CC000263A964206D39A7F2D2A03D2002801DA002034E0032832DDE28A019C2489A242A3
:201CE0002DD114468F3C082C02D9B83A082A26D8032024E0A0000020FFFF0000702000001B
:201D000000300040D0010020040A0A00DC050000F00300208020050000340040B80B00007A
:201D2000029ACA4E128AA48D9219944215D90A7C082A02D338682864A4E7521C0A74C3229E
:201D4000920098752A82A874002801D0012048710120087202F0CFF994E70022EEE700B5CD
:201D6000BB490C220A7415224A748874B94908208871B9480321C172012002F0BCF900BDC2
:201D800000B5B3490C220A7425224A74020A8A74C874B0490220887102F0ADF900BDAD483D
:201DA00010B52038007CFFF785FBC4B2A949A848621C1039113002F023F9A5480C21017417
:201DC000A44902208871204602F095F910BDA04810B52030417C0124491EC9B241748A0741
:201DE0009E48002A03DA818B2143818310BDCA079B49028B0BD08A430921090251180183A9
:201E000098488480018830229143018010BD8A431B210902511801838F4880228038018C22
:201E2000114301841046FEF739F98F4801782143017089486038C07A6028E7D18448052152
:201E40004038817210BDF8B581492031487C800702D0FFF7BCFFF8BD7F484030027F002A1D
:201E600002D0FFF755F9F8BD794A794E803A336C1268784D9C46D41A403D0E23EB5E9C42D0
:201E800003DB482132640177EBE7734C607A850705D5FD210840607202F0E2F9F8BDC50796
:201EA0000BD04A7D002A02D0521E4A7502E0400840006072FFF708F9F8BD410705D5FB212F
:201EC0000840607202F0C2F9F8BD614FBC21803FC9593F680507791A002D12DA642910DA42
:201EE0006546AA1AD218FF235F339A4209DDF72108406072564806214038817202F09EF928
:201F0000F8BD554D3022803D2B46403302400093002A6FD04F490B7A002B6CD000230B7215
:201F20004D49302A097A04D1CA0601D5202200E01022D706484A0123803A128C1343002FEF
:201F400035DA009F0022BA77102211432172A27A002A0CD0012A0FD0022A1DD0032A20D005
:201F6000EF221040607248084000207231E00020FFF706FF002012E03C4948780978000206
:201F8000084347BA3846FFF7FBFE012020737805400D001D20804BE0FFF701FF0220207377
:201FA00046E00520C002FFF7EBFE0320F7E7EF2739402172E77A002F11D0012F2BD0022F45
:201FC0002BD0032F2BD0DF2210406072FD2001402172012060732B84FEF760F828E088063F
:201FE00017D588070DD5E088A188884204D10120400202E017E019E0012002432A84FEF716
:202000004DF8607ADF2108406072207ADD2108402072FF2004E0002002E0552000E0332068
:20202000FFF79DFE04E0B06C814201DBFFF79FFD288EFEF7D7F800998988081A00D5404241
:20204000C82800DC5CE73220B064F8BD49020000B0010020300400208000002000300040D6
:20206000001F000000340040406C0040000800209204190CEA000D00140D0000965A845A18
:20208000963E963D963CA0281400000072B6DA480179FD2211400171D74962B6002020319C
:2020A0000870D6480121018003210180D549D4488880D548082181727047F8B5002105221B
:2020C0000846D201D04B4400403BE3189B181B8D401C59181028F5DB0803010CCB4CCC4A95
:2020E00048086186801802F065FA264640363081C548807A05287DD12046008EFEF772F858
:202100002146B080603100912546897B2C46C907E034C03500295BD1FEF7DDF8BA4F60378D
:20212000B87C022808D2F18A0905C90E052903D1298AFF3125312982A97F8008081806212A
:202140004843B049C01C8881B048408EFDF7C8FFB87C052805D2AF498A88920709D50122B9
:2021600006E0052805D9AB498A88920701D403228A80FEF795F8BA7C0B2A01D2002108E002
:202180000F2A01D2012104E0142A01D2022100E00321A0480388F026B34389010B4303801B
:2021A000297F891A00D500216A7F23794900D21851186983818802888901D20818231A4045
:2021C000008811434009062210400143009801738E482B8A878D90485E1F00210211B742F1
:2021E00019DA6356002B0EDB09D0462B0ADD5923DB4300E03FE023703C23EB7703E0E87FB7
:20220000401C207010466379002B27D061716178491C617022E06E8B21709B19BB4216D278
:20222000E97761797D48002904D1012161716178491C61707349898BBB22D200914211D962
:202240007D225201821A91420CD200230BE06E4940390978CB014B4059B208186949898B38
:202260009042E9D10C236B4A118A0C24A1431943118264498880F8BD10B5FEF709FA684879
:20228000FEF76AF8FFF719FF002010BD5E4900B564484039C8675D480F2120308177624974
:2022A000582008825E48FEF757F8604940200881FDF74CFF00BDFEB553480090877A52492A
:2022C0005248403102910146C0310A8A01924E4A868D403A1446A0341568627CE0303B0008
:2022E00002F092F90604162688884088D00604D4102002436274FFF7C9FF43484038006821
:202300001E2877D902F081F800980121817271E00120000385426DD93C484030C08A00054A
:20232000C00E052801D142480882029805645EE0930702D0FFF74BFD5CE0019B9E4206D241
:20234000029B1B6CEB1A7D25ED00AB4206DB07231A4362740022CA8442704BE0294835495E
:20236000818047E0334D019BA43D5D19324BAE4219D91D7CFA2D03D9224B81251D8001E036
:202380006D1C1D740023C356002B01D05B1C03701E4B4578E0331B79052D06D90025CD84AD
:2023A000457018330FE00025EBE7CD8C4B266D1CADB2F600CD84B54208D90025CD8445703B
:2023C000042B02D91B1F037100E0057150070CD5E07B401CC0B2E073FA2803D30020E073D0
:2023E00001F0EDFFFDF739FF04E0100702D40099022088720020FEBD00600040004400404F
:20240000BF5D000000380040700100200000002000DC050000340040DF2E00006F1700008F
:202420003C2400007922000000300040003C0040B6050000ED02000030040020121112037F
:2024400012111204F3041E08240109000F0DC30012300E0010B52D480022407A02280AD0AF
:20246000012808D0FF202A490130086029480272FEF7B0F807E02849C878030603D503072B
:2024800003D0401EC870002010BD24480274CA70F9E710B520480021C1702148012101805F
:2024A000812202801E4A8820203210711B4A4802403A90801B4810803020908117482038D0
:2024C0008183164B1981184C9480104C647A022C01D01C7410BD154B1383818181828180F3
:2024E00091830A210182018301810180FF210231818308487F218182402101720C4980158B
:20250000086003498039086010BD00006000002080E100E0406C0040700400204034004024
:2025200000380040F30A0000030200000550000080E200E0FC4910B50020C8640A46C867B5
:202540008032D0624031D0654887012353850B46022280335A83032240335A81087248727A
:2025600010BDF2491C208882F148A5210180002101757047ED48818A072212029143ED4AB7
:20258000137C1B0219438182517C08020843E7494039088188817047E7480621817240385B
:2025A00001688030C164E049C87A420702D5FB221040C872DF48007F002802D1DD49203193
:2025C000C870DE480122018C1203914301847047DB4A41088A1810B50146104601F0EAFF7C
:2025E000D6494031088110BDF0B5D449D54AC031084620308C8C80796043000A012393838D
:20260000497F002926D1CD4B6108C0331B7F884201D3002005E0CD1A081A2E1F864200D231
:20262000281F03256D03641EC64F2C43203F3C839C1C94818C1C1482022595821D19158380
:20264000851C5E1996804118891C1181BD83181800191080FF2002309083F0BD70B5044623
:20266000B1480021C173014620314879002804D0401E4871052C00DD0524B048B24A403005
:202680000188914205D20121C9438C4208DD0C4606E0AD4A5A32914202D2022C00DD022493
:2026A00022224188825EA548891A6030007808264843C511A148038E0246C91A128C00299A
:2026C0000ADC49420909491C3243494202844CB20820FDF7E3FC0AE098490822098C914335
:2026E000AB42018403D9002C01DD012407E0002C45D004DA61427F2902D97F2100E021464A
:202700008E4DC035AA8CE88A2B462033824219D98E4E8908715CFF26D536B24202D9012964
:2027200000D94908002C05DB5018A98A814205D2084603E04418944200D2501A80219971E4
:20274000A88417E0042901D8012200E04A089E79002C09DBB11880290BD980398908891C8F
:202760004018A884802104E0E97C8818B04200D2B11A9971FFF738FFA88CFFF729FF70BD06
:2027800030B46C4AD37D5B1CD375034620331C46DB7B0B43E373002101601046C038007B4D
:2027A000012828D81046A038007F012823D810466038007B01281ED810464038007F012821
:2027C00019D85D48807A04280AD0104620304278521C52B24270052A00DD417030BCDBE675
:2027E000D07D032807D9507F002804D13220507730BC052032E730BC70474F48062181721E
:20280000403801688030C1644A49002020314870704749484030407C411FC92900D3ECE7DA
:202820004649E031087270473F48407A010908290BD101074048090F4030C27C5207520F5F
:20284000914202D1417C8A0900D0D6E78A063B49920EA0318A71027D4031D30852078B7254
:20286000520F4A72344904228A72344A0021203291752D4A20329171E032517720329170AD
:2028800051702D4940390968C1630164704710B52548417AC02902D0FFF7AFFF10BD80211D
:2028A00041722549254808225131F83001F0A8FB10BD70B51C4C607A002802D0FFF79DFF62
:2028C00070BD1D481D4D4030417CE0356974408A294640BA20394886422803D115490120C6
:2028E000C03148731449154804225431F43001F087FB287D000601D5C02000E0802060727D
:2029000070BD0D4810B54030017C28292ED1427C803892211923095C5B01C0180C2A17D018
:20292000012A21D022E00000B00200206040004000740040B003002070010020000000208F
:2029400060EA000020340040B8100000303F000000290BD1F74902220A7400224A74817B9F
:2029600010221143817310BD002918D0F14C403C208C0004F7D4F048C17B042901D904212B
:20298000C173EC48CAB2ED49183001F039FB218C0120C00301432184FDF780FB10BDE64ACA
:2029A0004032D17B491CC9B2D1730329F6D2017E01221143017610BDF0B4E048062150388C
:2029C0008172DD4900236039FF304B704130C27A04242243C272FF38813802688030FF328F
:2029E000F532C264D34C407C203C0A46203AE076092803D2D24E4500755B5562012808D060
:202A0000CB785B1CDBB2CB70022B06D9082802D003E0CB7001E0CB485062E07A0A2801D005
:202A2000F0BC6EE7F0BC7047C24905220A744874C14810222030817B11438173BD480122CF
:202A40002030C17B1143C1737047F8B5BA48826D416D006D8918081A0D210907401801F0A8
:202A600009FCB5482030007B00280ED00421B148A030427A5118B14AF032127A511A00D587
:202A80002C31847A002C02D002E00521EFE70124081B00D52C300022A84E1546903E0AE05B
:202AA00083009B19C0331F8B5B8BBA185D19401C2C2800D300208842F2D12146104601F036
:202AC00079FD9C4E0746B0802146284601F072FD01469D48BB094843020C7809C018328050
:202AE00080183246403A90874F43F800C01B000BF8BDF8B591488F4D90380168803000903D
:202B00000164FF30012101300173A035687C112843D3E8787F2840D0FFF797FF29462039E7
:202B20008885074600982039407C89792C4648437D21C9004843060A603CA6871020205E16
:202B4000E17B381A4843642101F04AFD381A618A801B411A0320285628225043081A214645
:202B60002039097A022900D30020744990390A680099C96C511A754A91420EDD6E4B0024D0
:202B8000603B002808DD9878401CC0B29870032803D92720FFF748FF9C70F8BDFEB5674FF2
:202BA000F037B87A401C0006000EB87206D162496039C878002801D0401EC8705F4D5D4BE4
:202BC000503D2846403800682C4686464034607CA97A84465748A0334038008C564A0190F8
:202BE0001E46207C4032803E0093042904D002297ED003297DD012E17D218901F9824E4DEE
:202C00004C492035203903281ED004285BD02B461B7E02285AD005286CD00F2879D018287A
:202C200068D0192866D028287BD029287FD038287DD0012874D00628FCD05128FAD07128BA
:202C4000F8D08128F6D0EAE0112020568875404A0192002809DD9279521CD3B2019A192BC7
:202C6000937105D31923937102E0019B00229A7118228A56904209DB7078401CC0B2707027
:202C8000497E884204D34020FDF708FA002070702A4890380068E0630120F8730098017AF2
:202CA0000198C171287EC1070FD0400840002876204820494030027F0A74407F4874A87BF8
:202CC000102108432AE0FFF714FFA8E0507BC00774D06046C876062870D1E16C7046411A56
:202CE00014487D222030D200007A91420EDC04E046E066E01BE00CE013E0401CC0B23072E6
:202D0000022802D3012003432B7688E0022855D385E07046E063A87BF7210840A8737EE098
:202D200076E06046182802D1A07C012812D0FFF7E8FD74E04000002030040020C001002099
:202D4000503F0000FFFF000080B5010070170000D0020020102003432B76002090730A20D3
:202D6000C87201220198F549D20290430884FFF723FEF3480068E0642020FDF78FF94EE004
:202D8000012802D0022819D042E06046D871002078720321A972EB490B7C4C7C1B016408C0
:202DA00023430B75E74B714680339966009905230B7230725073D07331E0FFE7FFF7FCFDC6
:202DC0002DE071280AD0812813D0512814D0062815D0002815D005281AD912E0012001999D
:202DE000D64AC00201431184FDF758F9FFF761FD15E0FFF74CFD12E0FFF716FD0FE0FFF76B
:202E000008FD787A401CC0B201097872082902D0FFF7F3FC03E00007000F0728F8D80020F9
:202E2000FEBDC849087C072801D2401C08747047C449087C002801D0401E0874704730B5B1
:202E4000C04CFF23A289E1891520C333002520568A4208D9511AE574994208D9022804DDB1
:202E6000FFF7E6FF09E0E57403E0801C08E0642907D2811C03DAFFF7D4FF65750BE0801EC2
:202E8000607515202056002801DD401E02E0002801DA401C6075E17DA07D8900628B4018EF
:202EA000D108FF2800D9FF20884214D0884202D9637E5B4263761018401A6083607C617E50
:202EC0004018C0B26074022801D2022002E0202801D920206074A575E575FFF74BFB00204D
:202EE000A581C043E08130BD974900200880481596490860704700B5FFF7F6FF92491820C5
:202F00006031888200BD10B5FFF7F5FF9049812008809049002088804A158E4940398A80EE
:202F20000A8802239A430A808B498A8B520852008A83844A0A218032517281497F4AA031FF
:202F400008747E4940310881118C080504D5980281431184FDF7A2F810BDF0B5794F91B0B5
:202F60000D1E044611D03946C039201D0691032D16D0A278E9B2002A41D0072A3AD9402104
:202F80002046FFF7FDFB11B0F0BDB87D401CB8752078012801D90121F2E700202060F2E7A2
:202FA00001228A72A17800291FD0002121730D460226A178491EC9B2A1700B5C012B08D01A
:202FC000237B002B08D00023AD00AD1C2373B61C05E06D006D1C01E022736D00761C0029D6
:202FE000E7D1701C4008E07001E0002502260020207312E01154A078401CA070C3E7012D61
:203000000AD02078012821D0207B002823D0002001252073022600E001262078002802D0D4
:203020006078401C60704648617840300F9006297AD901203877786A002875D041480021CB
:20304000203041700F99062088729CE70120A07021710699F8E7012020730025DCE7E80758
:20306000C00F049020786D08761E002808D001282CD0022859D0032874D00020207047E18D
:20308000049800281FD06078401CC0B260700428F5D301202070F97C002904D1F874002063
:2030A000B881401EF8810B98C07A0A28E7D10898807B0028E3D10A981021007E08430A9983
:2030C000087600212DE00020607021E10498002804D060784128D2D902212AE003202070EE
:2030E0000021A1736173E173079841821448E2780068801A099A10650F9A927A022A02D18D
:20310000099A5438D0640B98C07A0A28B7D10898807B0228B3D20A981022007E10430A9A22
:20312000107608988173F3E0D6E00498002815D004212046FFF724FBEAE013E000000020C6
:2031400030010020B00300200040004080E100E0003800404034004000300040032020703B
:203160000020B7E0607B082809D2A07B0199049A415C4908D2011143019A8154A8E0082822
:2031800015D0049800287DD0A17B019AE07B8A5C5040E07300291FD0009A127B914272D109
:2031A000002859D010212046FFF7EAFA88E0A17B0198085C00F036FF01460498814201D030
:2031C000082182E0A07B002805D00099097B88427ED1012635467BE00E98807B400604D559
:2031E000F7480178402251400170207CFEF762F90099401C087302202070217C042904D106
:203200000799097B0143079801730B98C07A0A2856D1207C012853D10898807B022810D26D
:20322000FFF771FEFFF760FE069900208872E5480168099841650D9906200874079948739C
:203240003EE00B980821C1722020FCF727FFDD4801680C98816633E0FFF746FE06990020D3
:203260008872D8480168099841650D990620087407994873FFF7E3FDFFF75CF90098027BAB
:20328000D04801E020E019E09030019900F0B8FE0098017B0C98C17372B6CB4801F006F826
:2032A00062B60E98807B40060AD5C548027820214A40027002784A40027001E00220207063
:2032C000A07B401CA07303E020212046FFF758FA607B401C60731BE0BC480890BC480146A6
:2032E00060300E90B7482031A0300D90B7480B9140380C90204620300090B64807902046F3
:2033000010300190AF4880300990B04820380A90002E00D0A3E636E6F8B50520A94CC00187
:203320002618FF34C134207A617A884202D10020E072F8BDA848008AB289824200D2B08172
:20334000F289824200D9F08148009E4A491C8018FF308130058D0807000F9E4F60724C37E5
:2033600008E0680704D5A907890F3846FFF7F5FD2D093037002DD6D0F3E710B59648027808
:20338000037995494039087E0F240C769B07410804249B0F21401943930609019B0F0B430A
:2033A000014621401943130709019B0F0B434100214019430B019107890FC007854C1943BF
:2033C000400F08434034217A7E4A49008918FF3181310885207A401C0007000F2072E07A2B
:2033E000002806D17D4800F061FF002801D10120E07210BD00B5FFF79DF87A497848486212
:203400007549142020318882FFF7B4F872480822403802710D210172602101736E49203948
:203420000A71714A0A82714A8A82714A0A83714A8A83714A41151160704A1160FF210176AF
:203440006249C039897C01821021018000BD10B55F4901200A8C000302430A84FCF71EFEC8
:20346000FF205A49F53040394866002010BD70B5634E6520B080FFF7B7F8544C403CA07BEA
:20348000401CC1B24F48A173A030027E914206D9817E0025012910D000F0D5FDA573494817
:2034A000A17B8030C08EC840C207484948488039C030002A17D0098B16E003210174454896
:2034C0008573B58001204D4940028031086040496031C87BC20705D040084000C87349485E
:2034E00000F0E4FE70BD498A818470BDFEB53748384920380190807B002500285ED0314C39
:20350000C2062646920F8036A034002A2CD0327C042A53D0C10620460F38009000290CDA14
:203520002B484030007CFDF7C5FF29490746421C5031009800F064FD03E0707CFDF7BAFF71
:2035400007463574791C009800F063FD1D49C91980318874FF1C27736573A5736576022061
:20356000A07600F070FD0FE0C20701D0264806E0820701D5254802E040071DD52448F08632
:203580000F2020760120A0760198114B85730F48257440388573C0334038998C1A4641822F
:2035A000203AD4790222A507AD0FAA4092B2028364072FD589182EE0019885738D73FEBDBB
:2035C000406C0040300100209D2B00007004002000000020B0020020404000401933000054
:2035E0007B330000000100201D260000151D00000E1500002C10000080E200E000E100E025
:20360000403400404F34000055550000333300002D2D0000891A01839984FF49FD4848628E
:203620000120FE4940020860FD490860FD4905208880C4E78100FC4A091F89188B8DFB49C0
:203640008000001F8B858018C08DC8857047F8B5F748F6498446406D8039C001000CC8855D
:203660006046006DF34FC001000C8885397AEF4E8A00F149403E5118C0314883EF49484301
:20368000000CEF493080884201D2012005E0ED49884201D2022000E00320E44CE17E2546A1
:2036A000203D002906D06A7B824208D06873012903D004E0E07668730120FFF7BBFF6046C9
:2036C000416D806D09186046006D091A0091A18ADD4800F06FFF0099228B4843F188891ACC
:2036E000A27E514301229204891800F079FF2C21615EFF31FF3102314143C817C00D40182D
:203700002E21615E40120B1800D50023287A002402281ED3C648F18C4030994203DA018C0D
:20372000491C018400E00484B18C994203DA418C491C418400E04484018CC44A914203D85A
:20374000418CC34A914204D9048444843220FFF76BF958119911401831884118B3488038B3
:2037600081870386387A8100B3480818C0300383387A401CC0B238722C2800D33C72F8BD40
:2037800010B5FFF74EFBAA480821803841740121417600214183FEF7EDFE0020C043FEF7E7
:2037A0005DFF10BDAB4A90800020108190811082A84B012020331870002909D009211180DB
:2037C0001978C907FCD01080908A0005000D70471121F4E710B5A04881210180FF2181804B
:2037E000052101819D49818107220280018200240475FEF7F9FE8B49012008818948984952
:20380000403801809249EB398180302181818A48A0300474E0308473C47310BD10B58448A6
:20382000002101654165C165417A0422114341728C48FCF791FD10BD00B5FFF75CFB7E4863
:2038400005214030817200BDF8B578494039C889002876D00022CA81810602D5FDF732FA91
:203860006EE07349C30720318A7B002B01D0102002E0830703D5012002438A7360E06E4C51
:20388000430622468032009215222546520126684035A218B446002B17DA6448724B80384A
:2038A000018C4C0409D59943018400996046C8640620A8720020507042E019430184A87A3C
:2038C00004283DD1FFF7B8FF3AE00306584E002B27DA564F3346603FF87A4033082802D068
:2038E0000A2815D02CE0087E102210430876002098730A20F872FFF75FF800982168C164CA
:203900004A4801228038018CD2029143018417E00820F87200209873062050706046B0662A
:203920000EE0C0050CD5FFF7EEFA5048818B012211438183707AFD21084070720520A87285
:203940000020F8BDF0B53C4889B040300390817A3648374A203808903648603A4030079024
:203960003248354E40380590203801903248304D006800922D4A049260320692203A80361C
:20398000803D2C4C2A4F02920B0000F03DFE070520AFFEFDFCFB1F00787AC00710D1796D43
:2039A000386D1622411A0498825E8818B8650898C07B800705D50820787203980521817294
:2039C00075E12A48818B4908490081836CE10199C97A0929F4D00A2973D0F16C401A1E28E2
:2039E0005EDB02D12249102088820020214D009053E028780821084328700098401C009095
:203A0000052847DB00210520FFF7CCFE0599497B090131E06F3400000001002080E200E0CE
:203A200000E100E040340040404700008000002030040020B00200203001002080B501003D
:203A40006A1800003A200000B083850030750000EE0200000044004000380040FFFF000043
:203A6000F3090000283F0000004000000030004060400040003C00408142A1DA01980921D6
:203A8000C172FE482222018C114301841046FCF705FB0CE1142000F031FD28780007A8D458
:203AA000F748B96E0068F74A411A0498807B5043814203DB01204003FCF7F0FAFA2002E094
:203AC000FFE70298C07BEE49F26C09688A1A8242DFDBF16403980221817200206072A072F9
:203AE000E948818B012211438183E0E0607A002808D100210420FFF755FE0599C880607A25
:203B000000281FD0C0B2022860D0142871D0DC48F16C0068401A682854DB0198C07A0A283E
:203B20000FD0287F002807D000984078401C41B200980629417004DB0099002048706862CF
:203B4000287784E008980025457002980299008A888405997D2209889201914202D906996F
:203B60008A7B02E002998A7C06998A71FEF730FD079885720198C07A0A2824D1C3490A7EDD
:203B8000D30603E08BE0D4E069E058E008462030002B03DB817B491C817302E0EF231A407F
:203BA0000A76817B05290ED38573009806214170B3480068B86601990820C87241204001F3
:203BC000FCF76CFA37E0FFF705FE34E000990120085600280ED000216182297C4200491CFA
:203BE0008907890F2974697C80180818C006C00E0EE014E000206883012068760198C07A10
:203C00000A2809D0287D4106490F00072974C00E6874FEF7A6FC0EE00498C07FF3E7787ADB
:203C2000FD2108407872FFF7E5FB9448008C400401D5FFF701FE607A401C607237E0079928
:203C4000897A002906D0316D401AAA282FDBFEF7A3FC24E0716D401A1628F8DA27E0316C0A
:203C60008B4A874B411A914205DB217B03290FD1002121733064F16B864A411A91421DDB4C
:203C80000098C078401CC1B200980A29C17002D8FEF782FC01E0FEF7B0FD1868B866FFF725
:203CA00032F906990020C871039901208872E07A40084000E072002009B0F0BD697F00295F
:203CC00001D0491E6977E18A002908D0491E0904090CE18203D10146FF3978393165316D3C
:203CE000FF22411A7832914202DB3065FFF748FD607B002808D00121401E0006A173000E9B
:203D0000607301D1FFF7F2FB6348C1790029CED0491E0906090EC171C9D1A17B002902D0FF
:203D20000121C171C3E7019916200856FEF796FCBDE70006000EBAD1FEF787FEFEF754FCCE
:203D40000298808CFEF744FCB1E770B54E4802212030018049496031497A032906D05A21DE
:203D60000180FFF7D0F8FCF735FC48E0474D203D687A082802D14948FCF7EEFA40480126C7
:203D8000A030017C0446E03400290ED0491E0906090E017409D1A17B002902D1E17B0029F8
:203DA00001D0067401E0FFF725FBE07AC00708D172B63B4800F07AFA002802D1E07A3043F0
:203DC000E07262B62E480078800704D1687A400701D4FFF73CFC686E002810D0401E6866F9
:203DE0000DD1264809212030C1722038018C2022114301841046FCF751F9FEF7FEFC002028
:203E000070BDF8B50120274940028880411E1E480182818B01221143818323490183FCF73B
:203E2000F2FD1948132520300580422101731B49124820223C31D03000F0FEF80F48154946
:203E40004030C8390246418073232032137096224284E12292008284AF229200C284044671
:203E600006224034A27364222282E573618201467F2220390A764A766E2217E00000002004
:203E80003001002060EA00000030004050040020D8590000A4060000D0020020283F00006F
:203EA00045390000003400407B1B0000427319480025184F8572403F1748FD677860174868
:203EC000B86708467D22A030C273C038828C144B08261A438284CE72018C202211430184F3
:203EE0001046FCF7DBF80F4938683A4688668032FA38D0640A2048720846803860394562FE
:203F00004D70057446740F218174A17F0175FFF785FCF8BD700100204B3D00004938000030
:203F200002380000300400200203020302030504010204070C0E10121416181A1C1E1F20BC
:203F40002122232425262728292A2B2C2D2E2F3000006900D200B80B00000000FFFF0000DD
:203F60000000000096018033120296010000000005000000000000500000000000000000F7
:203F800000004C00FFFFFFFFFFFFFFFFFFFFFFFFFFFFFFFFFFFFFFFFFFFFFFFFFFFFFFFFF1
:203FA000FFFFFFFFFFFFFFFFFFFFFFFFFFFFFFFFFFFFFFFFFFFFFFFFFFFFFFFFFFFFFFFF21
:203FC000FFFFFFFFFFFFFFFFFFFFFFFFFFFFFFFFFFFFFFFFFFFFFFFFFFFFFFFFFFFFFFFF01
:203FE000FFFFFFFFFFFFFFFFFFFFFFFFFFFFFFFFFFFFFFFFFFFFFFFFFFFFFFFFFFFFFFFFE1
:00000001FF
